S02300002E5C2E2E5C62696E5C64656D6F70726F675F73746D3332663035312E73726563B9
S3150800200000200020992C0008EB2C0008ED2C000875
S3150800201000000000000000000000000000000000B2
S31508002020000000000000000000000000EF2C00087F
S315080020300000000000000000F12C0008C52E000872
S31508002040F72C0008F92C0008FB2C0008FD2C0008CA
S31508002050FF2C0008012D0008032D0008052D000897
S31508002060072D0008092D00080B2D00080D2D000866
S315080020700F2D0008112D0008132D0008152D000836
S31508002080172D0008192D00081B2D00081D2D000806
S315080020901F2D0008212D0008232D0008252D0008D6
S315080020A0272D0008292D00082B2D00082D2D0008A6
S315080020B02F2D0008312D0008332D0008352D000876
S315080020C0EE11AA5510B5064C2378002B07D1054BFF
S315080020D0002B02D0044800E000BF0123237010BD86
S315080020E03C01002000000000A0300008084B10B595
S315080020F0002B03D00749084800E000BF07480368DB
S31508002100002B00D110BD064B002BFBD09847F9E7F2
S315080021100000000040010020A03000083C0100201B
S3150800212000000000164B002B00D1144B9D464022A0
S3150800213092029A1A924600218B460F461348144A71
S31508002140121A00F093FF0F4B002B00D098470E4B46
S31508002150002B00D098470020002104000D000D48F0
S31508002160002802D00C4800E000BF00F059FF20000C
S31508002170290000F07BFD00F03DFFC0460000080086
S315080021800020002000000000000000003C010020A4
S31508002190B4010020000000000000000080B500AF78
S315080021A0BFF34F8F024B034ADA60BFF34F8FFEE748
S315080021B000ED00E00400FA0580B500AF00F014F861
S315080021C0C046BD4680BDC04680B500AF00F06AF87F
S315080021D0C046BD4680BDC04680B500AFFFF7DEFFEE
S315080021E0C046BD4680BDC04680B588B000AF8023D6
S315080021F09B020121180000F08BFB80239B02012122
S31508002200180000F065FB9023DB0501220221180067
S3150800221000F0D8F99023DB0501220321180000F00D
S31508002220D1F91823FB180C221A601823FB1803226D
S315080022305A711823FB1802221A711823FB18002258
S315080022409A711823FB180122DA711823FA189023B9
S31508002250DB051100180000F0FDF83B00E122120230
S315080022601A603B0000225A603B0000229A603B003D
S315080022700022DA603B0000225A613B000C221A61F8
S315080022803B00074A1900100000F062FB044B0121CD
S31508002290180000F017FCC046BD4608B080BDC04611
S315080022A00044004080B500AF264B1B78002B16D1A2
S315080022B0254B180000F04EF80300012B3FD1224BA6
S315080022C01B78002B3BD000F0F3FD02001F4B1A6071
S315080022D01C4B01221A701E4B00221A702FE01C4B51
S315080022E01B785A1C184BD318180000F033F8030053
S315080022F0012B19D1164B1B780133DAB2144B1A701D
S31508002300114B1A78124B1B789A4218D10D4B0022A2
S315080023101A700D4B5B78FF2B11D10B4B9B78002B5A
S315080023200DD1FFF759FF0AE000F0C2FD0200074B86
S315080023301B6864339A4202D9024B00221A70C046BF
S31508002340BD4680BD580100205C010020A001002088
S31508002350A401002080B582B000AF78600B4B202125
S31508002360180000F0DBFB0300012B09D1074B18000E
S3150800237000F0C6FB0300DAB27B681A70012300E09E
S3150800238000231800BD4602B080BDC0460044004088
S3150800239080B582B000AF80231B030121180000F02E
S315080023A097FA3B00802292001A603B0001221A71BC
S315080023B03B0000229A713B0003225A713B0000221F
S315080023C0DA713B00074A1900100000F043F8802331
S315080023D09B00044A1900100000F0E4F8C046BD4608
S315080023E002B080BD0008004880B582B000AF00F09A
S315080023F05FFD03007B60144B1B687A68D21AF423CE
S31508002400FF339A421CD9114B1B78002B0AD10F4B6C
S3150800241001221A7080239B000D4A1900100000F053
S31508002420B1F809E0094B00221A7080239B00084A7C
S315080024301900100000F0B6F8034B7A681A6000E03D
S31508002440C046BD4602B080BDA8010020AC010020F0
S315080024500008004880B586B000AF78603960002370
S315080024607B6100233B610023FB6000237B6181E0E5
S3150800247001227B699A4013003B613B681B683A69F5
S315080024801340FB60FA683B699A4270D13B681B7936
S31508002490012B03D03B681B79022B38D17B689B68DC
S315080024A07A695200032191400A00D2431A407B6898
S315080024B09A607B689A683B685B7919007B695B0060
S315080024C099400B001A437B689A607B689B889BB28D
S315080024D07A691204120C012191400A0092B2D24381
S315080024E092B213409AB27B689A807B689B889BB2AB
S315080024F01AB23B689B7919007B691B041B0C99402F
S315080025000B001BB213431BB29AB27B689A807B6896
S315080025101B687A695200032191400A00D2431A4087
S315080025207B681A607B681A683B681B7919007B69A7
S315080025305B0099400B001A437B681A607B68DB686E
S315080025407A691204120C5200032191400A00D24300
S315080025501A407B68DA607B68DA683B68DB791900C1
S315080025607B695B0099400B001A437B68DA607B69DC
S3150800257001337B617B690F2B00D879E7C046BD46DE
S3150800258006B080BD80B582B000AF78600A00BB1C7B
S315080025901A80BB1C1A887B689A61C046BD4602B081
S315080025A080BDC04680B582B000AF78600A00BB1C0B
S315080025B01A807B68BA1C12881A85C046BD4602B0C6
S315080025C080BDC04680B584B000AF786008001100B1
S315080025D0BB1C021C1A807B1C0A1C1A700023FB6099
S315080025E00023BB607B1C1A78BB1C1B8807210B4089
S315080025F09B009A401300FB60BB1C1B88DB089BB240
S315080026001800BB1C1B88DB089BB21A007B680832C3
S315080026109200D358BA1C128807210A4092000F214B
S3150800262091400A00D2431A4011007B680200083222
S315080026309200D150BB1C1B88DB089BB21A007B6832
S3150800264008329200D258FB681343BB60BB1C1B8838
S31508002650DB089BB21A007B6808329200B968D15031
S31508002660C046BD4604B080BD80B588B000AF78606E
S315080026700023BB6100237B6100233B610023FB60D1
S315080026800023BB600023FB618A4B5B680C22134066
S31508002690BB61BB69042B0CD002D8002B05D03BE0EC
S315080026A0082B0AD00C2B33D036E07B68824A1A6096
S315080026B036E07B68804A1A6032E07E4B5A68F0231F
S315080026C09B0313407B617B4B5A68C0235B02134014
S315080026D03B617B699B0C02337B613B69002B04D110
S315080026E07B69764A5343FB610EE0724BDB6A0F2225
S315080026F013400133FB60F9686F4800F0EFFB0300F5
S315080027001A007B695343FB617B68FA691A6007E024
S315080027107B686B4A1A6003E07B68674A1A60C046A2
S31508002720644B5B68F0221340BB61BB691B09BB6144
S31508002730644ABB69D3181B78DBB2BB607B681A682E
S31508002740BB68DA407B685A605A4B5A68E023DB005C
S315080027501340BB61BB691B0ABB615A4ABB69D318E4
S315080027601B78DBB2BB607B685A68BB68DA407B685B
S315080027709A60504B1A6B80235B00134003D17B6829
S31508002780514ADA6010E04B4B5A688023DB0113404C
S3150800279005D17B689B685A087B68DA6004E07B6829
S315080027A09B689A087B68DA60424B1B6B4022134091
S315080027B003D17B68454A1A6103E07B6880221202CE
S315080027C01A613C4B1B6B1022134003D17B683A4AB3
S315080027D05A6103E07B681A687B685A61354B1B6B44
S315080027E00322134004D17B689A687B689A611EE0CD
S315080027F0304B1B6B03221340012B04D17B681A68EC
S315080028007B689A6113E02B4B1B6B03221340022B48
S3150800281004D17B68802212029A6108E0254B1B6B63
S3150800282003221340032B02D17B68234A9A61214B6A
S315080028301A6BC0239B02134004D17B689A687B6895
S31508002840DA6127E01B4B1A6BC0239B021A408023D0
S315080028505B029A4204D17B681A687B68DA6119E0E0
S31508002860144B1A6BC0239B021A4080239B029A4280
S3150800287004D17B6880221202DA610BE00D4B1A6BD9
S31508002880C0239B021A40C0239B029A4202D17B684E
S31508002890094ADA61074B1B6B8022134003D17B6818
S315080028A0074A1A6202E07B68FA691A62C046BD46A0
S315080028B008B080BD0010024000127A0000093D00F1
S315080028C0006CDC02C0000020809FD500128000004A
S315080028D080B582B000AF78600A00FB1C1A70FB1C3A
S315080028E01B78002B06D0094B084A51697A680A43B7
S315080028F05A6106E0054B054A52697968C9430A4098
S315080029005A61C046BD4602B080BDC04600100240AE
S3150800291080B582B000AF78600A00FB1C1A70FB1CF9
S315080029201B78002B06D0094B084AD1697A680A43F6
S31508002930DA6106E0054B054AD2697968C9430A4057
S31508002940DA61C046BD4602B080BDC04600100240EE
S3150800295080B58EB000AF7860396000237B630023B2
S315080029603B630023FB627B681B68012293431A00C2
S315080029707B681A607B685B68FB62FB6A4B4A13409C
S31508002980FB623B689B68FA6A1343FB627B68FA6AD8
S315080029905A607B681B68FB62FB6A454A1340FB6208
S315080029A03B685A683B68DB681A433B681B691343F4
S315080029B0FA6A1343FB627B68FA6A1A607B689B684B
S315080029C0FB62FB6A3B4A1340FB623B685B69FA6A37
S315080029D01343FB627B68FA6A9A600823FB1818009F
S315080029E0FFF742FE7B68344A934204D10823FB185A
S315080029F09B693B630CE07B68304A934204D1082309
S31508002A00FB18DB693B6303E00823FB189B683B6301
S31508002A107B681A6880231B02134014D03B6B5A004C
S31508002A203B681B681900100000F058FA03007B6326
S31508002A303B6B5A003B681B681900100000F0D4FA7B
S31508002A400B00FB6210E03B681B681900386B00F04E
S31508002A5045FA03007B633B681A683B6B1100180054
S31508002A6000F0C2FA0B00FB623B681B685A08FB6A57
S31508002A709A4202D87B6B01337B637B681A68802392
S31508002A801B0213400AD07B6B5B0807221340FB62CC
S31508002A907B6B0B4A1A40FB6A13437B637B6B9AB2C8
S31508002AA07B689A81C046BD460EB080BDFFCFFFFF4A
S31508002AB0F3E9FFFFFFFCFFFF003801400044004038
S31508002AC0F0FF000080B582B000AF78600A00FB1CFA
S31508002AD01A70FB1C1B78002B06D07B681B6801222A
S31508002AE01A437B681A6006E07B681B6801229343D9
S31508002AF01A007B681A60C046BD4602B080BDC04653
S31508002B0080B582B000AF78607B689B8C9BB2DB0592
S31508002B10DB0D9BB21800BD4602B080BD80B584B0FF
S31508002B2000AF786039600F23FB1800221A707B68A3
S31508002B30DB693A68134004D00F23FB1801221A7088
S31508002B4003E00F23FB1800221A700F23FB181B78CB
S31508002B501800BD4604B080BD80B500AF1B4B1B4AAC
S31508002B60126801210A431A60184B184A5268184914
S31508002B700A405A60154B154A126816490A401A60E7
S31508002B80124B124A126814490A401A600F4B0F4A30
S31508002B90526812490A405A600C4B0C4AD26A0F21F5
S31508002BA08A43DA62094B094A126B0D490A401A63CD
S31508002BB0064B064A526B01218A435A63034B00228D
S31508002BC09A6000F00FF8C046BD4680BD001002406E
S31508002BD00CB8FFF8FFFFF6FEFFFFFBFFFFFFC0FF85
S31508002BE0ACFEFFFF80B500AF1D4B11221A601D4BCE
S31508002BF01C4A52685A601B4B1A4A52685A60194B4B
S31508002C00184A526818490A405A60164B154A5268BB
S31508002C10A02189030A435A60124B124A126880217E
S31508002C2049040A431A60C0460E4B1A6880239B045F
S31508002C301340F9D00B4B0B4A526803218A435A605A
S31508002C40084B084A526802210A435A60C046054B97
S31508002C505B680C221340082BF9D1C046BD4680BDDF
S31508002C600020024000100240FF7FC0FF80B500AF81
S31508002C7000F008F8FFF7A0FAFFF7B6FBFFF7A4FA8B
S31508002C80FAE7C04680B500AFFFF782FB00F0ECF824
S31508002C90C046BD4680BDC04608498D460849094A12
S31508002CA0094B9B1A05DD00240859105104349C422F
S31508002CB0FADB064880470648004700000020002047
S31508002CC0AC300008C00000203C010020592B000849
S31508002CD0252100081849194A002301E00B60043130
S31508002CE09142FBD3FFF7C2FFFEE7FEE7FEE7FEE7EA
S31508002CF0FEE7FEE7FEE7FEE7FEE7FEE7FEE7FEE79E
S31508002D00FEE7FEE7FEE7FEE7FEE7FEE7FEE7FEE78D
S31508002D10FEE7FEE7FEE7FEE7FEE7FEE7FEE7FEE77D
S31508002D20FEE7FEE7FEE7FEE7FEE7FEE7FEE7FEE76D
S31508002D30FEE7FEE7FEE700003C010020B4010020A4
S31508002D40B0B582B000AF02003960FB1D1A70FB1DDA
S31508002D501B787F2B32D92F4CFB1D1B781A000F23AB
S31508002D601340083B99082B4AFB1D1B7818000F23B4
S31508002D700340083B9B0806339B00D31804331B68A3
S31508002D80FA1D1278100003220240D200FF2090405C
S31508002D900200D2431A403B689B01FF201840FB1DE6
S31508002DA01B781D0003232B40DB00984003001A43C1
S31508002DB08B1D9B00E31804331A6027E0164CFB1D95
S31508002DC01B785BB29B081449FA1D127852B2920816
S31508002DD0C03292005258F91D0978080003210140B3
S31508002DE0C900FF2088400100C94311403A68920192
S31508002DF0FF201040FA1D1278150003222A40D2003F
S31508002E00904002000A43C0339B001A51C046BD4693
S31508002E1002B0B0BD00ED00E000E100E080B582B090
S31508002E2000AF78607B680E4A934201D9012312E00D
S31508002E300C4B7A681202120A013A5A6001235B4265
S31508002E4003211800FFF77CFF064B00229A60054B0A
S31508002E5007221A6000231800BD4602B080BDC0468E
S31508002E60FFFFFF0010E000E080B500AF084B1A68CE
S31508002E70FA239900100000F031F803001800FFF754
S31508002E80CDFF002000F006F8C046BD4680BDC0460E
S31508002E90D000002080B582B000AF7860034B7A6816
S31508002EA01A60C046BD4602B080BDC046B0010020CB
S31508002EB080B500AF024B1B681800BD4680BDC046F2
S31508002EC0B001002080B500AF034B1B685A1C024BAB
S31508002ED01A60C046BD4680BDB001002000224308E6
S31508002EE08B4274D303098B425FD3030A8B4244D3C4
S31508002EF0030B8B4228D3030C8B420DD3FF22090206
S31508002F0012BA030C8B4202D31212090265D0030BC4
S31508002F108B4219D300E0090AC30B8B4201D3CB03BA
S31508002F20C01A5241830B8B4201D38B03C01A5241FC
S31508002F30430B8B4201D34B03C01A5241030B8B42FE
S31508002F4001D30B03C01A5241C30A8B4201D3CB02E9
S31508002F50C01A5241830A8B4201D38B02C01A5241CE
S31508002F60430A8B4201D34B02C01A5241030A8B42D1
S31508002F7001D30B02C01A5241CDD2C3098B4201D3E9
S31508002F80CB01C01A524183098B4201D38B01C01A67
S31508002F90524143098B4201D34B01C01A52410309DE
S31508002FA08B4201D30B01C01A5241C3088B4201D38D
S31508002FB0CB00C01A524183088B4201D38B00C01A3A
S31508002FC0524143088B4201D34B00C01A5241411A61
S31508002FD000D20146524110467047FFE701B500206E
S31508002FE000F006F802BDC0460029F7D076E770471C
S31508002FF07047C046084B10B50400002B02D00021CC
S3150800300000E000BF054B1868836A002B00D098477C
S31508003010200000F033F8C046000000009C3000088D
S315080030200E4B70B500251E000D4CE41AA410A542DF
S3150800303004D0AB00F35898470135F8E700F020F8BC
S31508003040084B00251E00084CE41AA410A54204D01B
S31508003050AB00F35898470135F8E770BD34010020F6
S3150800306034010020340100203801002003008218B2
S31508003070934202D019700133FAE77047FEE7000061
S31508003080F8B5C046F8BC08BC9E467047F8B5C046B9
S31508003090F8BC08BC9E46704743000000D4000020D8
S309080030A0000000001E
S30D080030A480F0FF7F0100000027
S315080030AC00000000010203040102030406070809D4
S315080030BC006CDC02000000000000000000000000AC
S315080030CC00000000000000000000000000000000E6
S315080030DC0000000098300008000000000000000006
S315080030EC00000000000000000000000000000000C6
S315080030FC00000000000000000000000000000000B6
S3150800310C00000000000000000000000000000000A5
S3110800311C00000000ED200008C520000897
S70508002000D2
